:020000040000FA
:040000006B303A28FF
:08000800A000030EA100831209
:1000100005191028831601178312B23081002B288E
:1000200083160113831203140B190310A80DA90DD5
:10003000AA0DAB0DAC0DAC16FF302C02031D2B2806
:10004000FA302B02031D2B2831152A08AF0029088E
:10005000AE002808AD008B100B11210E8300A00EFE
:04006000200E090065
:0C007400203084008001840A6030040207
:10008000031C3C281230B00090218316FF239000FF
:10009000831283160C308505870183128501870141
:1000A000073099000030831691008312C830831600
:1000B0008100831231309000003083168C0083124F
:1000C00010308B00831600309B001C141A0883121A
:1000D000BC00831610309B001C141A088312BD004C
:1000E000D42181018E018F010B118B100B108C011B
:1000F0008B17882031198B20B30B862803108519A4
:100100000314B90DF030390203191721ED217928B4
:1001100064003210080031110130B7008B13203019
:10012000370783169B001C141A088312A400103092
:10013000370783169B001C141A088312A300A6001D
:100140000230A6060030370783169B001C141A08DD
:100150008312A200A7000130A7068B17321CB62815
:1001600022090339A200A309A409A50924082F0222
:10017000031D112923082E02031DE52822082D0244
:10018000031D112901303702031DC9283D143E14F7
:100190009D2102303702031DD028BD143E14A12139
:1001A00003303702031DD7283D153E14A521043026
:1001B0003702031DDE28BD153E14A9210530370284
:1001C000031DE5283D163E14AD2126082E02031D11
:1001D000112927082D02031D112901303702031DA3
:1001E000F4283D103E14B12102303702031DFB28D4
:1001F000BD103E14B52103303702031D02293D1105
:100200003E14B92104303702031D0929BD113E14E3
:10021000BD2105303702031D10293D123E14C121B6
:100220001129B70A06303702031808008E2801305A
:10023000B600B300B400B500B70085018701B11363
:100240008820B30B4329031085190314B90DF0302E
:10025000390203196A29B40B432901303702031903
:10026000C521023037020319C821033037020319B0
:10027000CB21043037020319CE2105303702031990
:10028000D1219630B400311D20293111321C4D2965
:100290002D090339AD00AE09AF092F1C20298E01AD
:1002A0008F010C1C20290C102E1E20298B132030AE
:1002B0003707BB002F08BA007D2110303707BB007D
:1002C0002E08BA007D2100303707BB002D08BA0088
:1002D0007D218B1785018701B70AB60106303702E9
:1002E000031C2029D42108003E1C08003E101030B9
:1002F000BB003D08BA007D2108008B133A08831625
:100300001C159A003B089B0055309D00AA309D00AB
:100310009C1464009C1889291C1183128B170800F7
:10032000FF30D000D415D515D615D715D815D91549
:10033000DA15DB15DC15DD150800D2104E14CE10D1
:100340000800D2114E15CE110800D2124E16CE1250
:100350000800D2134E17CE130800D3104F14CF103D
:1003600008005210CE144E1008005211CE154E1136
:1003700008005212CE164E1208005213CE174E131A
:1003800008005310CF144F100800303085060800C5
:1003900003308506080006308706080021308706EE
:1003A00008001830870608003D184E143D1CCE1476
:1003B000BD184E15BD1CCE153D194E163D1DCE1651
:1003C000BD194E17BD1DCE173D1A4F143D1ECF143B
:1003D0004E08D200CF00D30008008F080319080090
:1003E0008F01D00F2F2BD00A521C052A541DFB2938
:1003F000D4015416132AD41D002AD4015416132AEA
:10040000541E132AD401D414132AD41C0A2AD4014A
:100410005415132A541D0F2AD401D415132A541E1F
:10042000132AD4015415D21C242A551D1A2AD50189
:100430005516322AD51D1F2AD5015516322A551EAA
:10044000322AD501D514322AD51C292AD5015515B1
:10045000322A551D2E2AD501D515322A551E322A8B
:10046000D5015515521D432A561D392AD601561657
:10047000512AD61D3E2AD6015616512A561E512AF9
:10048000D601D614512AD61C482AD6015615512A0F
:10049000561D4D2AD601D615512A561E512AD6016F
:1004A0005615D21D622A571D582AD7015716702A91
:1004B000D71D5D2AD7015716702A571E702AD701FB
:1004C000D714702AD71C672AD7015715702A571DD1
:1004D0006C2AD701D715702A571E702AD7015715D5
:1004E000521E812A581D772AD80158168F2AD81DE6
:1004F0007C2AD80158168F2A581E8F2AD801D81462
:100500008F2AD81C862AD80158158F2A581D8B2A65
:10051000D801D8158F2A581E8F2AD8015815D21EF7
:10052000A02A591D962AD9015916AE2AD91D9B2AEF
:10053000D9015916AE2A591EAE2AD901D914AE2AAC
:10054000D91CA52AD9015915AE2A591DAA2AD901A3
:10055000D915AE2A591EAE2AD9015915521FBF2AE4
:100560005A1DB52ADA015A16CD2ADA1DBA2ADA013D
:100570005A16CD2A5A1ECD2ADA01DA14CD2ADA1CEF
:10058000C42ADA015A15CD2A5A1DC92ADA01DA1508
:10059000CD2A5A1ECD2ADA015A15D21FDE2A5B1D3A
:1005A000D42ADB015B16EC2ADB1DD92ADB015B16A2
:1005B000EC2A5B1EEC2ADB01DB14EC2ADB1CE32AB1
:1005C000DB015B15EC2A5B1DE82ADB01DB15EC2A5D
:1005D0005B1EEC2ADB015B15531CFD2A5C1DF32A14
:1005E000DC015C160B2BDC1DF82ADC015C160B2BE6
:1005F0005C1E0B2BDC01DC140B2BDC1C022BDC0146
:100600005C150B2B5C1D072BDC01DC150B2B5C1E1A
:100610000B2BDC015C15D31C1C2B5D1D122BDD018B
:100620005D162A2BDD1D172BDD015D162A2B5D1EA5
:100630002A2BDD01DD142A2BDD1C212BDD015D15AC
:100640002A2B5D1D262BDD01DD152A2B5D1E2A2B95
:10065000DD015D1574214E08D2004F08D30050080B
:10066000D1000C305405031D05120C305505031D37
:1006700085120C305605031D05100C305705031D5F
:1006800085100C305805031D87100C305905031DCB
:1006900007110C305A05031D07100C305B05031DB4
:1006A00087120C305C05031D07120C305D05031D1D
:1006B000871151080E020318892B12305405031DAF
:1006C000051612305505031D851612305605031DFB
:1006D000051412305705031D851412305805031DEB
:1006E000871412305905031D071512305A05031DD2
:1006F000071412305B05031D871612305C05031DBD
:10070000071612305D05031D8715FF3050020319CF
:1007100008008F08031D0800882051080E02031CE2
:10072000892B18305405031D051206305405031D8E
:10073000051618305505031D851206305505031D95
:10074000851618305605031D051006305605031D85
:10075000051418305705031D851006305705031D75
:10076000851418305805031D871006305805031DE1
:10077000871418305905031D071106305905031D4C
:10078000071518305A05031D071006305A05031DBA
:10079000071418305B05031D871206305B05031D27
:1007A000871618305C05031D071206305C05031D13
:1007B000071618305D05031D871106305D05031D02
:0407C0008715080091
:084000000200030002000600AB
:02400E00CC01E3
:10420000010078007A007C007E007B0079007F004E
:104210007D007A0078007E007C00FF00FF00FF0038
:104220000000F200F600FA00FE00F200F600FA00CC
:10423000FE00F200F600FA00FE00FF00FF00FF00A3
:10424000010005000500050005000900090009003E
:1042500009000D000D000D000D00FF00FF00FF0024
:10426000FF00FF00FF00FF00FF00FF00FF00FF0056
:10427000FF00FF00FF00FF00FF00FF00FF00FF0046
:10428000FF00FF00FF00FF00FF00FF00FF00FF0036
:10429000FF00FF00FF00FF00FF00FF00FF00FF0026
:1042A000FF00FF00FF00FF00FF00FF00FF00FF0016
:1042B000FF00FF00FF00FF00FF00FF00FF00FF0006
:1042C000FF00FF00FF00FF00FF00FF00FF00FF00F6
:1042D000FF00FF00FF00FF00FF00FF00FF00FF00E6
:1042E000FF00FF00FF00FF00FF00FF00FF00FF00D6
:1042F000FF00FF00FF00FF00FF00FF00FF00DD00E8
:00000001FF
